:100000000C9434000C9451000C9451000C94510049
:100010000C9451000C9451000C9451000C9451001C
:100020000C9451000C9451000C9451000C9451000C
:100030000C9451000C9451000C9451000C945100FC
:100040000C9451000C9451000C9451000C945100EC
:100050000C9451000C9451000C9451000C945100DC
:100060000C9451000C94510011241FBECFEFD4E02A
:10007000DEBFCDBF11E0A0E0B1E0EAE6F3E002C0F0
:1000800005900D92AA30B107D9F721E0AAE0B1E0BE
:1000900001C01D92AB32B207E1F70E9464010C94DB
:1000A000B3010C94000088E18093C10086E0809346
:1000B000C2001092C50083E38093C400089590911C
:1000C000C00095FFFCCF8093C6000895CF93DF93C7
:1000D000EC018991882319F00E945F00FACFDF912B
:1000E000CF910895CF93DF93CDB7DEB727970FB6A3
:1000F000F894DEBF0FBECDBF4AE0BE016F5F7F4FF9
:100100000E947E01CE0101960E94660027960FB6DE
:10011000F894DEBF0FBECDBFDF91CF910895CF938E
:10012000DF93CDB7DEB727970FB6F894DEBF0FBECB
:10013000CDBF42E0BE016F5F7F4F0E947E01CE01C6
:1001400001960E94660027960FB6F894DEBF0FBE98
:10015000CDBFDF91CF910895CF93DF93CDB7DEB7B9
:1001600027970FB6F894DEBF0FBECDBF40E1BE01AA
:100170006F5F7F4F0E947E01CE0101960E94660054
:1001800027960FB6F894DEBF0FBECDBFDF91CF919B
:1001900008958AE00C945F008091C00087FFFCCF37
:1001A0008091C60008951F93CF93DF930E94CC00E7
:1001B000CAE0D1E01C2F105E8A3041F0882331F074
:1001C0001C1721F089930E94CC00F6CF18828AE098
:1001D00091E0DF91CF911F9108958AB1806E8AB925
:1001E0008091000181FF03C08BB18F718BB9809129
:1001F000000180FF03C08BB1806E8BB9089580939E
:10020000000108950C94ED00482F8091000181FFBA
:100210000BC09BB121E030E0042E01C0220F0A94F4
:10022000EAF7209529232BB98091000180FF0AC0AD
:100230005BB121E030E0C90101C0880F4A95EAF7BF
:10024000852B8BB908959091000191FF0AC09BB155
:1002500021E030E0082E01C0220F0A94EAF7292B92
:100260002BB99091000190FF0DC04BB121E030E01F
:10027000B90102C0660F771F8A95E2F7CB0180951E
:1002800084238BB90895CF93C82F0E9423018FE157
:100290009EE40197F1F700C000008C2F0E9404013A
:1002A0009FEF2AE683E0915020408040E1F700C0B4
:1002B0000000CF91089585E00E94430186E00E94EE
:1002C000430187E00C94430182E00E94FF000E94FA
:1002D00002010E9453000E945B0181E091E00E94B4
:1002E000660085E00E9443012FEF89E698E12150E6
:1002F00080409040E1F700C00000EFCFBB274A30BC
:1003000031F4992322F4BDE2909581959F4F0C948E
:100310008A01BB27FB015527AA27880F991FAA1F0F
:10032000A41710F0A41B83955051B9F7A05DAA3310
:1003300008F0A95DA193009779F7B111B1931192DB
:10034000CB010C94A301DC01FC01672F7191772391
:10035000E1F7329704C07C916D9370836291AE1780
:0A036000BF07C8F30895F894FFCF1B
:0A036A000152454144590A00000009
:00000001FF
